:1000000018308A0000280000FF00030E8301A100C1
:100010000A08A0008A010408A2007708A300780853
:10002000A4007908A5007A08A6007B08A70083131E
:1000300083128C308400801E1F288C1A39288B1E56
:1000400023280B193628220884002308F7002408E7
:10005000F8002508F9002608FA002708FB00200808
:100060008A00210E8300FF0E7F0E09008A110A12FA
:10007000C32A8A110A12CD2A0A108A100A1182078D
:1000800028340C34013406340A108A100A1182070D
:100090000A3400340E3411341F3411341134003456
:1000A000043400340E3411341F341134113400344C
:1000B000043400340E3401340F3411340F3400345E
:1000C00004340E3415340434043404340434003459
:1000D000043404340434043415340E340434003449
:1000E0000034003400340034003400340034003470
:1000F0000034003400340034003400340034003460
:10010000003400340034003400340034003400344F
:100110000A108A100A118F3E03188A0A820041349D
:1001200001342F344234013406344334013447342B
:100130004434013430344534013409344634013414
:10014000423447340234323448340234343449348B
:10015000023436344A34023438344D34E234003414
:100160004E34E23402344F34E23404345034E23456
:1001700006345134E23408345234E2340A3453340D
:10018000E2340C345434E2340E34583401344E34F6
:10019000593401344F345A34013450344B34E1343F
:1001A00010344C34013453345534E2342034313477
:1001B000E13415343234E13416343334E234173454
:1001C0003434E13419343534E234223436340234F0
:1001D00051343734E2341A343834E2341C3439348C
:1001E000E2341E346134023444346234E134253460
:1001F0006334E13424346434E23426346534013425
:1002000007346634013449346734E13428346834BF
:10021000E23429346934E2342B346A3402346234EF
:100220000A148A100A1182070034003400340034A2
:1002300000340034013400341C34E234003400341F
:10024000443404343C3400342834F1340034003471
:1002500001340034013400341534E1340A340034FC
:1002600063340034013400341634E1340134003492
:100270005A3400340134003416340234013400346A
:1002800001340034013400340A148A100A11820740
:100290000C34563469347234683465343A3420345A
:1002A0004B346134743474342E340A346C34753401
:1002B00075346B346B3475342F3459346C34693481
:1002C0006B34753475346D3400340A148A100A1195
:1002D00082070C3441346A346134733474346934C1
:1002E0006E3400340A148A100A1182070C34563412
:1002F00069347234683465343A34203450346534A7
:100300006C346C3465347434743469340A346C3449
:100310006F3470347034753400340A148A100A1142
:1003200082070C34563469347234683465343A3494
:1003300020344C34693465346B346B346934E434C0
:100340000A346534693420346E34E43468347434E7
:10035000793400340A148A100A1182070C34563496
:1003600069347234683465343A34203459346C3426
:1003700069346C34E4346D347034F63400340A1467
:100380008A100A1182070C34563469347234683486
:1003900065343A34203453346134763475346134FE
:1003A00000340A148A100A1182070C345634693456
:1003B0007234683465343A34203453347934F63442
:1003C00074347434F6340A346D3469346E346934F8
:1003D0006D34693473347334E43400340A148A108D
:1003E0000A11F53E03188A0A82000C345634693427
:1003F0007234683465343A3420340A3454347534F1
:100400006E34743465346D34613474346F346E34E6
:1004100000340A108A140A1182070C344B34E43475
:1004200079346E347434693461342E342034253494
:100430006C3475343A3425343034323475342034E5
:100440000A3453347934F63474347434F634203442
:100450002534643420342534253420342534633461
:1004600000340A108A140A118207543461346C343F
:100470006C3465346E346E34653474346134613494
:100480006E3400340A108A140A1182070C34413485
:100490006A3461347334743469346E3420346134B2
:1004A000723476346F3400340A108A140A118207C9
:1004B000543475346E346E346934743400340A1034
:1004C0008A140A1182070C3441346A34613473345B
:1004D000743469346E342034283431343D34533428
:1004E000653469347334293400340A108A140A11CB
:1004F00082070C344D34613478342E3473347934BB
:10050000F63474347434F63400340A108A140A1140
:1005100082070C344D3469346E342E34733479349C
:10052000F63474347434F63400340A108A140A1120
:1005300082070C344C34E4346D347034F634743443
:1005400069346C3461340A3425346C3464342034B6
:1005500025346334433400340A108A140A118207A4
:10056000503465346C34323431345F34563465344D
:1005700072345F3432342E34303436340A344634F4
:1005800069346E340034B10BC82A3C140130B10018
:10059000BD170B118A110A12232818088316DF00D1
:1005A0005F080339003A0319E62A83121A088316F2
:1005B000DF0083121A088316DF0083121A088316DD
:1005C000DF00831218121816FD2A831610308312CA
:1005D0006507F800640878020F39F6007608F8001D
:1005E00078080E3C031CFD2A6630650784001A0853
:1005F0008000013065070F39E5008C128A110A125C
:100600002328D630840000080319152B0130F80088
:10061000F701F70B092BF80B082B4A30F700F70B03
:100620000F2B00000000800B062B003483165D0E9C
:10063000F039F7000F3083120805770488000000B6
:10064000081400000000081000348810F0308316F1
:100650008800831208150000081400000808080E1E
:100660000F398316DD008312081000000814000003
:100670000808080E0F398316DC00831208100030BA
:10068000831688005D0EF700F030F70577085C04EC
:10069000F8007808DC00DC1F4F2B8312262B5A1839
:1006A000542B8312881083165A1C592B83128814DA
:1006B00083160000831208110000081083165B0ED9
:1006C000DC000F30DC055C08DD0083121623831686
:1006D0005B080F39DC00DD00831216230034003084
:1006E0008316880083128810081108100F308316B3
:1006F000D6008312012301308316C3004308033C54
:10070000031C8E2B0330DD00831216230530831665
:10071000D600831201238316C30A7E2B0230DD002C
:10072000831216238316C3014308033C031CA52B25
:10073000430883123C208316C400DA014408DB001E
:10074000831225238316C30A942B0530D600831207
:1007500001238316C30143083F3C031CC62B4030D2
:100760004307C400DA014408DB0083122523831603
:100770004308831244208316C4000130DA00440881
:10078000DB00831225238316C30AAB2B83128A1541
:100790000A168D2883165508831203178D008316B9
:1007A0008C130C1483120C080313A9002908F800F9
:1007B000003483165308831203178D008316031326
:1007C0005408831203178C0083168C130C158312A4
:1007D00003130B138B138B1BEA2B55308316031754
:1007E0008D00AA308D008C14C030831203138B044B
:1007F000831603170C11831203130D1A022C831690
:100800000317FB2B0D12003483164E08D3004F083C
:10081000D4008312D923013083164E07D100D03083
:1008200084000008D2005108D3005208D40083127B
:10083000D923003483165008D5008312CA238316A7
:10084000D2017808D100D230D30001305007D40053
:10085000D5008312CA2383165308840078088000C9
:100860005108F8005208F900831200343D1F972CFC
:100870003D130330D5009330D4004E08053C0318D7
:10088000972C4E08073C031C972C60086104031941
:10089000522C60080319E103E00B522CE108031D00
:1008A000522CD7141A308316D00083121A247908D8
:1008B0008316C6007808C500013045078312DE00A4
:1008C000831646088312DF000318DF0A1A308316E6
:1008D000CE0083125F088316D00083125E08831651
:1008E000CF00831204241C308316D00083121A24F4
:1008F00079088316C4007808C30043084404031928
:10090000952C440883125F02031C932C031D902C2A
:100910005E0883164302031C8F2C8312932C8312D0
:10092000C9148430C600972C83168312C910003472
:10093000BD1D9E2C3D1D9E2C2F149F2C2F10E8308A
:100940008316890083120914831689008312091003
:100950008316890083120914300893008316141833
:10096000B32C8312AE2C83121308C700E830831611
:100970008900831209102F08930083161418C22CC3
:100980008312BD2CE83089008312891483168900F4
:10099000831289100608F038BF0040083F0203198F
:1009A000D62C40083F06C1063F08C0000034AF11F6
:1009B000B010BD110E308316D00083121A247908AE
:1009C000B9007808B8000230B500AE30B400B30109
:1009D000B201903083168700831207150930CE00CC
:1009E000D30100348316560858068039DA00D61F22
:1009F000FE2CD509D609D50A0319D60AD81F052D0C
:100A0000D709D809D70A0319D80AF801F901F7015B
:100A1000FA015808031D0F2D57080319292D10300E
:100A2000D9000310D50DD60DF70DFA0D58087A022E
:100A3000031D1C2D57087702031C252D5708F702AC
:100A4000031CFA035808FA020314F80DF90DD90B28
:100A5000112D0000DA1F312DF809F909F80A0319E0
:100A6000F90A8312003410308316D800F701FA0116
:100A7000D50CD40C031C422D5608F7070318FA0AAC
:100A80005708FA07FA0CF70CF90CF80CD80B382DAC
:100A900083120034F801F901F701FA0183165608B0
:100AA000031D552D550803196F2D1030D700031065
:100AB000D30DD40DF70DFA0D56087A02031D622DE1
:100AC00055087702031C6B2D5508F702031CFA0327
:100AD0005608FA020314F80DF90DD70B572D000034
:100AE0008312003420308316D00083121A24790830
:100AF0008316C9007808C8001530D5008312CA23B0
:100B000078088316CA001630D5008312CA237808E5
:100B10008316CB002430D5008312CA2378088316AD
:100B2000CC002530D5008312CA2378088316CD0067
:100B30002630D00083121A2479088316CF00780853
:100B4000CE0032304802F7004908FA000030031C9A
:100B50000130FA027708F8007A0883124502031C74
:100B6000BF2E031DB72D440878020318BF2E44087A
:100B700083164802F7004908FA0083124508031C4F
:100B8000450FFA0277088316C6007A08C70047089F
:100B9000FA004608C71FD52D4608003CF700FA01A9
:100BA0004708031C470FFA027708D0007A08D100E3
:100BB000D11BE12DD108031DA52E5008FE3C031CBE
:100BC000A52E4708FA004608C71FEF2D4608003C2F
:100BD000F700FA014708031C470FFA027708D00014
:100BE0007A08D100D11BFB2DD108031D272E5008F8
:100BF000273C031C272E46088312E2070318E30A4A
:100C0000831647088312E307E31B152E63082D3C68
:100C10000318152EFF3A031D112E6208E03C03183D
:100C2000152E2E30E300E030E200E31F252E63088E
:100C3000D13C031C252E031D212E62081F3C031CE2
:100C4000252ED130E3002030E2002A2E83168312B5
:100C5000E301E20163088316D6008312620883165B
:100C6000D5004F08D8004E08D7008312F224780828
:100C70008316C6070318C70A7908C707FA014C0884
:100C8000D0007A08D1004708D5004608D4005108A2
:100C9000D7004C08D6008312332579088316D2007A
:100CA0007808D100FA014D08D3007A08D400520820
:100CB000D6005108D5005408D8004D08D70083123B
:100CC000F22479088316C7007808C6004608323C2B
:100CD000C6004708031C470F6F2E0030702E003CE3
:100CE000C700FA014A08F800FA1F792EC71F852E9F
:100CF0007B2EC71B8B2E7A084702031C8B2E031DED
:100D0000852E4608780203188B2EFA014A08C60081
:100D10007A08C700A42EFA014B08F800C71F932ECB
:100D2000FA1F9F2E952EFA1BA42E47087A02031C49
:100D3000A42E031D9F2E780846020318A42EFA0144
:100D40004B08C6007A08C700BD2EC71BB42EC708C3
:100D5000031DAE2E4608003C0318B42EFA014B08C2
:100D6000C6007A08C700B92EFA014A08C6007A08F8
:100D7000C7008312E301E2018316C92E8312FA0130
:100D800083164B08C6007A08C7008312E301E2010C
:100D9000831646088312D30022308316D0008312B4
:100DA0001A2479088316C5007808C40083123D1CF4
:100DB000032F19308316D5008312CA238316D1015D
:100DC0007808D000FA01831253088316D2007A08FB
:100DD000D3005108D5005008D4005308D70052085A
:100DE000D6008312332579088316D2007808D10003
:100DF0005208D4005108D300D6016430D5008312C4
:100E00004A257808D300FA0153088316D0007A08DF
:100E1000D1004508D5004408D4005108D700500837
:100E2000D6008312332579088316D2007808D100C2
:100E30005208D4005108D300D6016430D500831283
:100E40004A257908D2007808D10000348316550865
:100E5000F801540203182F2F5408F7003B2FF70115
:100E60000830D600D40DF70D550877020318F700A7
:100E7000F80DD60B322F831200348316570B412FF7
:100E8000442F4030D800452FD80101305602D807F2
:100E900058088038D900DA015908DB00831225236D
:100EA0000034831655080C3A83120319702F063A42
:100EB00003197C2F023A0319842FEC3A03198B2F64
:100EC000013A0319932F133A03199B2F323A03194E
:100ED000A32F013A0319AA2F133A0319B12FB92FDF
:100EE0008316DA010130DB008312252302308316DA
:100EF000D60083120123C12F01308316D6000230A1
:100F0000D70083123D27C12F8316DA011030DB0092
:100F100083122523C12F01308316DA00E130DB0074
:100F200083122523C12F01308316DA000230DB0043
:100F300083122523C12F01308316DA00EF30DB0046
:100F400083122523C12F01308316DA00DB018312BF
:100F50002523C12F01308316DA00DB0083122523FD
:100F6000C12F01308316DA00EF30DB008312252316
:100F7000C12F01308316DA005508DB0083122523C8
:100F8000C12F0034F701F80183164C0803104D18E7
:100F9000F707F70CF80CCD18F707F70CF80C4D19FC
:100FA000F707F70CF80CCD19F707F70CF80C4D1AEA
:100FB000F707F70CF80CCD1AF707F70CF80C4D1BD8
:100FC000F707F70CF80CCD1BF707F70CF80C83129A
:100FD00000340C1EE92F83164C088312990000344C
:0C0FE00083164408CC008312E92700347B
:1010000004088316D4004E0EF038D000D007E23E1C
:10101000D100323ED3004E080F39D107D107D30794
:10102000E93ED200D207D2074D0E0F39D207D307BF
:10103000D20DD30DD309D30D4D080F39D307D00DE1
:101040000730CF000A30D307D203031C2328D2076E
:10105000D103031C2728D107D003031C2B28D0075A
:10106000CF03031C2F28CF308400073054055413BE
:101070008407D3300402031954170008F700031D36
:101080004928541B4928541A5928D4194928203072
:101090004C28D41554123030F707CE010408CD0087
:1010A0007708D5008A11831251278A1583164D08B7
:1010B0008400840A541F392883128A150A12352C99
:1010C000780883164D08D4006430D5008A11831245
:1010D00026278A1577088316CD0078083030031D3F
:1010E0007828CE1C8328CE1983284E1A20307B28DE
:1010F000CE114E124E14F8077808D5008A118312CB
:1011000051278A1583164D08D4000A30D5008A115C
:10111000831226278A1577088316CD007808303089
:10112000031D9828CE19A0284E1CA0284E1A203046
:10113000F8077808D5008A11831251278A1583167B
:101140003030CD074D08D5008A11831251278A15FA
:101150008A150A12432C203083164F1E3030D000DF
:101160004E08F700CE1FBB28F709F70A7708CE0014
:101170002D30D000CF174E08D4006430D5008A112E
:10118000831226278A1577088316CE003030780719
:10119000D1004E08D4000A30D5008A1183122627C8
:1011A0008A15303077078316D30030307807D200A5
:1011B0005008F700CF1DDE28CF1F4F114F1AEB2824
:1011C000CF1F06294F1906297708D100CF18062905
:1011D0007708D200062930305102031D062977080E
:1011E000D1002030D000CF1DF9284F11CF14CF1FD0
:1011F000CF1030305202031D06297708D20020306C
:10120000D100CF1DF928CF10CF1F4F104F1D0F2930
:101210005008D5008A11831251278A158316CF1CD6
:1012200018295108D5008A11831251278A1583166F
:101230004F1C21295208D5008A11831251278A1583
:1012400083165308D5008A11831251278A158A15EF
:101250000A12602C04088316D100CB1F3729D1173E
:10126000511ED10ACA09CB09CA0A0319CB0A4B0E6F
:10127000F038CD00CD07E23ECE00323ED0004B0824
:101280000F39CE07CE07D007E93ECF00CF07CF07F3
:101290004A0E0F39CF07D007CF0DD00DD009D00D92
:1012A0004A080F39D007CD0D0730CC000A30D007DF
:1012B000CF03031C5729CF07CE03031C5B29CE079E
:1012C000CD03031C5F29CD07CC03031C6329CC305D
:1012D000840007305105511384035105031D7729FC
:1012E000511A840A511A77292030F700942984076B
:1012F000D0300402031951170008F700031D882994
:10130000511B8829511AA029D119882920309329E5
:10131000D11F90292D30F70084035113D113942944
:10132000D11551123030F707CB010408CA007708F5
:10133000D5008A11831251278A1583164A08840022
:10134000840A511F782983120034831644080B3C09
:10135000031DB5291A30CE00D001CF018A118312A6
:1013600004248A15DF01DE0183164408083C031DAE
:10137000C52A0130831248078316CA00D4000630FC
:10138000D5008A11831226278A1577088316C6008E
:10139000460DF700F70DF70DF830F7057708013E19
:1013A0008A11831210218A15F8008316C700470896
:1013B000DF3C0318C52A460DF700F70DF70DF8308E
:1013C000F7057708043ECA004A0A8A1183121021E1
:1013D0008A15FA0083164A088A11831210218A1589
:1013E000DA007A08DB008316460DF700F70DF70DDB
:1013F000F830F7057708023ECA004A0A8A118312BC
:1014000010218A15FA0083164A088A1183121021C6
:101410008A15DC007A08DD008316460DF700F70D0B
:10142000F70DF830F70577088A11831210218A1515
:10143000F8008316C8004708E13C031D4B2A480802
:10144000D5008A118312CA238A1578088316C90029
:10145000460DF700F70DF70DF830F7057708063E53
:10146000CB004B0A8A11831210218A15FA008316C9
:101470004B088A11831210218A158316CC00490863
:10148000D4004C08D5008A11831226278A15D90169
:101490007808D80083164708E23C031D842A4808D0
:1014A000D0008A1183121A248A1579088316CA007B
:1014B0007808C900460DF700F70DF70DF830F7056D
:1014C0007708063ECC004C0A8A11831210218A1537
:1014D000FA0083164C088A11831210218A1583168C
:1014E000CD007A08CE004A08D4004908D3004E083F
:1014F000D6004D08D5008A1183124A258A1579082D
:10150000D9007808D80083164708EF3C0318A32AAF
:101510004808D5008A118312CA238A1578088316D1
:10152000C90047080739F8004908F700F808031907
:101530009D2A0310F70CF80B992A770801398312BA
:10154000D800D901831683125B085902031CB22A02
:10155000031DAE2A58085A020318B22A5B08D900A4
:101560005A08D80059085D02031CC02A031DBC2A72
:101570005C0858020318C02A5D08D9005C08D8002E
:101580005714BB019830BA00831644080A3C031D67
:10159000F72A8312C908031DCF2A8316F72A0130C0
:1015A000F7004A08F8000319D92A0310F70DF80BC1
:1015B000D52A7708FF3AC905BB010230BA004A08AC
:1015C000FB3E0318F62A053EAF2EF62A1A30831684
:1015D000CE00D001CF018A11831204248A15DF01C5
:1015E000DE01F62AC201F62A3D12F62A83164408C5
:1015F000453C031D812C831257104E080B3C031DE4
:101600000B2B49084B05003A031D0B2BCE01BC13D5
:101610003C13D001CF01C9080319E62B8316C5017D
:101620004508073C031CE42B8312CA0A0730CA058D
:101630004908F7004A08F8000319222B0310F70C99
:10164000F80B1E2B771CE12B4A08F83E0318DA2B07
:10165000083EB82E8316C90149088A118312442115
:101660008A158316C90AF700D5008A1183125127FB
:101670008A151C3083164902031D2C2B8312DA2B8A
:101680008316C90149088A11831265218A158316B8
:10169000C90AF700D5008A11831251278A1508302C
:1016A00083164902031D422B8312DA2B8316C901CC
:1016B00049088A11831272218A158316C90AF70014
:1016C000D5008A11831251278A15163083164902D4
:1016D000031D582B8312DA2B8316C90149088A117E
:1016E00083128D218A158316C90AF700D5008A1145
:1016F000831251278A15183083164902031D6E2B59
:101700008312DA2B8316C90149088A118312AA2190
:101710008A158316C90AF700D5008A11831251274A
:101720008A15103083164902031D842B8312DA2B8D
:101730008316C90149088A118312BF218A158316AD
:10174000C90AF700D5008A11831251278A150D3076
:1017500083164902031D9A2B8312DA2B8316C901C3
:1017600049088A118312D1218A158316C90AF70004
:10177000D5008A11831251278A1518308316490221
:10178000031DB02B8312DA2B8316C90149088A1175
:101790008312EE218A158316C90AF700D5008A1133
:1017A000831251278A15133083164902031DC62B55
:1017B0008312DA2BC801BB012D30BA008316E42B4B
:1017C00083128316C50A102B812C83123F08F93C23
:1017D000031DF52B1A308316CE00D001CF018A11DC
:1017E000831204248A15DF01DE015F088316D4000A
:1017F00083125E088316D300D6013C30D5008A11CF
:1018000083124A258A1579088316CA007808C90008
:1018100083125F088316D40083125E088316D300F8
:10182000D6013C30D5008A1183124A258A157708E3
:101830008316CB00CC014C088A11831209228A1529
:101840008316CC0AF700D5008A11831251278A1516
:101850000A3083164C02031D1B2C103084004A08EA
:10186000CE004908CD00831200283A308316D500F7
:101870008A11831251278A1583164B08CD00013037
:10188000CE008312602812308316CD004D088A11D5
:10189000831209228A158316CD0AF700D5008A1112
:1018A000831251278A151B3083164D02031D462CC7
:1018B000831253088316CE001F30CF008312AB284B
:1018C00020308316D5008A11831251278A152530BE
:1018D0008316D5008A11831251278A15203083166A
:1018E000D5008A11831251278A154D088316D50019
:1018F0008A11831251278A15C801BB010F30BA0023
:1019000083164408093C031D852D831257188A2C21
:101910008316852D5710480DF700F70DF70DF83099
:10192000F7057708013E8A1110218A15F800831601
:10193000C7008312480DF700F70DF70DF830F705D3
:1019400077088A1110218A15F8008316C800470805
:10195000E13C031DDA2C8312480DF700F70DF70D5B
:10196000F830F7057708063E8316CA004A0A8A113E
:10197000831210218A15FA0083164A088A118312ED
:1019800010218A158316CB00831258088316CC00C9
:101990004B08CD008A118312C2278A157808831656
:1019A000CC004808D3004C08D4008A118312D923F4
:1019B0008A1583164708E23C031D192D8312480D32
:1019C000F700F70DF70DF830F7057708063E831698
:1019D000CA004A0A8A11831210218A15FA00831656
:1019E0004A088A11831210218A158316CB007A08BF
:1019F000CC00831259088316D50083125808831629
:101A0000D4004C08D7004B08D6008A118312332526
:101A10008A1579088316CD007808CC004808CE00D6
:101A20004D08D0004C08CF008A11831204248A1577
:101A300083164708EF3C0318562D4808D5008A1135
:101A40008312CA238A1578088316C5008312D80822
:101A500003193C2D831647080739C9000130F700E8
:101A60004908F8000319382D0310F70DF80B342D31
:101A70007708C5044D2D8312831647080739C9001E
:101A80000130F7004908F80003194A2D0310F70D3B
:101A9000F80B462D7708FF3AC5054808D3004508DE
:101AA000D4008A118312D9238A1583168312C801A0
:101AB00001308316D6000230D7008A1183123D27E9
:101AC0008A158316C90149088A11831231228A15A1
:101AD0008316C90AF700D5008A11831251278A1587
:101AE0000C3083164902031D632D0330CA002E30CB
:101AF000D5008A11831251278A158316CA0B772DB8
:101B00008312BB010F30BA00831683124808FA3ED5
:101B10000318AC2E063EC42E83164408083A8312DE
:101B2000031DC62D8316C90149088A11831242225A
:101B30008A158316C90AF700D5008A118312512726
:101B40008A150D3083164902031D942D0A30D600E4
:101B50000230D7008A1183123D278A158316C901E6
:101B600049088A11831254228A158316C90AF7007C
:101B7000D5008A11831251278A150630831649022F
:101B8000031DB02D01308312C800C62DAC2E831664
:101B90004408083A8312031DE52D8316C90149083C
:101BA0008A1183125F228A158316C90AF700D500AD
:101BB0008A11831251278A15113083164902031D99
:101BC000CF2D02308312C800E52DAC2E83164408B9
:101BD000083A8312031D222E8316C90149088A116F
:101BE000831275228A158316C90AF700D5008A1157
:101BF000831251278A150B3083164902031DEE2DDF
:101C000003308312C8000A308316D6000230D70092
:101C10008A1183123D278A1525308316D5008A1133
:101C2000831251278A1520308316D5008A1183121A
:101C300051278A1520308316D5008A118312512727
:101C40008A15222EAC2E83164408083A8312031DEF
:101C50005F2E8316C90149088A11831285228A15CD
:101C60008316C90AF700D5008A11831251278A15F5
:101C70000B3083164902031D2B2E04308312C8003B
:101C80000A308316D6000230D7008A1183123D270E
:101C90008A1525308316D5008A11831251278A159B
:101CA00020308316D5008A11831251278A152030DF
:101CB0008316D5008A11831251278A155F2EAC2E08
:101CC00083164408083A8312031D9E2E0530C8006F
:101CD0008316C90149088A11831295228A15831631
:101CE000C90AF700D5008A11831251278A150B30D3
:101CF00083164902031D6A2E1030840083124508A2
:101D00008316CB00831244088316CA0083122A214B
:101D100020308316D5008A11831251278A15DF30AF
:101D20008316D5008A11831251278A1543308316F2
:101D3000D5008A11831251278A159E2EAC2E831648
:101D40004408083A8312031DAB2EC8015710BB018B
:101D50000230BA00AB2EAC2E8A110A16FA2A0A10EB
:101D60008A140A158207E52AE62AF32AF22AF42AB7
:101D70000A108A140A1582072A2B402B562B6C2B2B
:101D8000822B982BAE2BC42B0A108A140A158207BB
:101D90008C2DC72DE62D232E602E9F2E20308316EE
:101DA000C4008A118312F0278A1556308316C400A6
:101DB0008A118312F0278A158316C30143088A11FA
:101DC0008312AC228A158316C30AF700C4008A1155
:101DD0008312F0278A15123083164302031DDE2E6C
:101DE0000D30C4008A118312F0278A1500343D1586
:101DF000320833040319042F32080319B303B20B5A
:101E0000042FB3080319BC14340835040319102F28
:101E100034080319B503B40B102FB50803193C158A
:101E20003608370403191C2F36080319B703B60BFD
:101E30001C2FB7080319BC15380839040319282FBB
:101E400038080319B903B80B282FB90803193C1631
:101E50003A083B040319342F3A080319BB03BA0BA1
:101E6000342FBB080319BC16540855040319402F1E
:101E700054080319D503D40B402FD50803193D1777
:101E8000D6080319442FD6038A150A163D2A663050
:101E9000640784000008FC0083168C120130831252
:101EA00064070F39E40083168C167C08F80083124F
:101EB0008A150A16442A83164508393C031C652FE7
:101EC00030304502F8006A2F6A2F4508DF39C93ED5
:101ED000F8006A2F831200348316CB1B832F0F3038
:101EE000F7004A0EF7050A30770203187A2F3030D0
:101EF000F7077C2F4B08F7077708CC008A1183126D
:101F0000E9278A1583160F30CA050A304A020318DA
:101F10008B2F30308D2FCB134B08CA074A08CC00CB
:101F20008A118312E9278A1500348316C908031D14
:101F3000A32F4608AB004708AC004808AD00831249
:101F4000D716CF2F8316C9080319D02F8312D71A9B
:101F5000AB2F8316D02F20308316CC008A1183122A
:101F6000E9278A1583162B08CC008A118312E927EA
:101F70008A1583162C08CA003730CB0083126C27D1
:101F800083162D08CA003730CB0083126C270D3022
:101F90008316CC008A118312E9278A15D71283167B
:041FA0008312003474
:102000008316430F19288312B301B201B501B4013D
:10201000B701B601B901B801BC103C11BC113C12AA
:10202000BC133C13BD10CE01D001CF01CC01162B47
:10203000831683124C08003A03192228013A031927
:1020400031284728491483164308853C031D2F284F
:1020500001308312CC004910CE01D30183168312C4
:10206000472883164308053C031D45288312CC01ED
:102070000B30CE00AF01B001903083168700831281
:102080000711BD114914D301831683124728500844
:10209000003A03194F28013A03195A286228831677
:1020A0004308813C031D582801308312D000831659
:1020B000831262288316430B60288312D001831693
:1020C000831262284F08003A03196A28013A03195B
:1020D00075287F2883164308023C031D73280130AE
:1020E0008312CF00831683127F2883164308823C15
:1020F000031D7D288312CF01831683127F284E088B
:10210000F13E0318F32A0F3E172B4B084905003AFE
:1021100003198D280B30CE00F32A4F0BB0284C0B3F
:10212000B028BD1EB0288316D0010A1283121A24CB
:102130000A167908B3007808B200AF15AF16AF14CD
:10214000AF172F152F162B308316D0000A128312CB
:102150001A240A167908E1007808E0000130CE0060
:10216000F32A83164308413A83120319BB28C33A62
:102170000319D228D728AF11AF12B01490308316AC
:10218000870083120715BD150A308316D0000A1286
:1021900083121A240A167908B5007808B4000230B0
:1021A000CE00D7280A12D7240A16AF12D728F32A4E
:1021B000500BE8281E308316D0000A1283121A240E
:1021C0000A167908B5007808B4000330CE00F32A67
:1021D00083164308423A83120319F228C03A0319BE
:1021E0000A290F29BD11B010AF1190308316870056
:1021F00083120711AF120C308316D0000A1283121B
:102200001A240A167908B3007808B200C20A083006
:10221000CE000F290A12D7240A16AF120F29F32A6B
:1022200083164308423A831203191A29C03A031944
:102230003229362990308316870083120715B01093
:10224000BD1104308316D0000A1283121A240A1614
:102250007908B5007808B40004308316AA00831208
:10226000CE0036290A12D7240A163629F32A8316F5
:102270004308423A831203194129C03A03196029DD
:102280006529AF168316AA0B53290630D0000A120F
:1022900083121A240A167908B5007808B4000530AC
:1022A000CE00652983160230D0000A1283121A2448
:1022B0000A167908B5007808B4000C30CE006529FC
:1022C0000A12D7240A16AF126529F32A8316430887
:1022D000423A831203197029C03A03197F298429CD
:1022E000AF1208308316D0000A1283121A240A167D
:1022F0007908B5007808B4000430CE0084290A12A9
:10230000D7240A16AF128429F32A83164308423AC7
:10231000831203198F29C03A031999299D29AF11F6
:10232000AF12B301E430B200B014BD150E30CE00D0
:102330009D290A12D7240A169D29F32A83164308D9
:10234000423A83120319B129013A0319B429C73A51
:102350000319D529063A0319D629833A0319DA292C
:10236000F1293D10C201F129AF110A1272250A1696
:1023700022308316D0000A1283121A240A16790812
:102380008316C5007808C4008312510883164402DE
:102390008312B600831645088312B7005208031C47
:1023A000520FB7020730CE00F129F1290A12D724C3
:1023B0000A16F129D301AF119030831687008312DA
:1023C0000711AF120C308316D0000A1283121A24A0
:1023D0000A167908B3007808B200C20A0830CE00A5
:1023E000F129F32A83164308423A83120319052A76
:1023F000013A0319082AC73A0319102A063A0319A1
:10240000112A833A0319152A2C2A3D10C2012C2ABD
:10241000AF155208B7005108B6000630CE002C2A7E
:102420002C2A0A12D7240A162C2AD301AF11903075
:102430008316870083120711AF120C308316D00069
:102440000A1283121A240A167908B3007808B20017
:10245000C20A0830CE002C2AF32A83164308413AD8
:102460008312031D522A4F0B4A2A10308316D500BF
:102470000A128312CA230A167808420203184A2A4B
:10248000BD1E4A2AAF16AF15B5019830B4000A3008
:10249000CE00512AC915AF10AF132F112F120B30D8
:1024A000CE00522AF32A83164308413A83120319B5
:1024B000602A033A0319662A063A0319702A812A08
:1024C00090308316870083120715812A9030831677
:1024D0008700831207110A30B300BA30B200812A94
:1024E000AF1290308316870083120711AF10AF131D
:1024F0002F112F122F17B5015B30B4000D30CE0015
:10250000812AF32A83164308423A8312031D9F2A25
:102510000A308316D0000A1283121A240A16790888
:10252000B5007808B400AF11AF12B014BD159030EB
:1025300083168700831207150230CE009F2AF32AE4
:10254000831643080A3A8312031DA72AA72AF32AEF
:1025500083164308423A8312031DB12A2F13CE017A
:10256000B12AF32A83164308413A83120319BC2A7D
:10257000C33A0319EE2AF22AB010BD11500BD82A23
:10258000AF15AF163D1417308316D0000A12831210
:102590001A240A167908B5007808B4000A127225C0
:1025A0000A165208B7005108B6000630CE00ED2AD0
:1025B000AF1190308316870083120711AF120C30D1
:1025C0008316D0000A1283121A240A167908B3005F
:1025D0007808B200C20A0830CE00F22A0A12D724C4
:1025E0000A16F22AF32A83164308C4000A128A152F
:1025F0008312A5290A168A11C90803190B2B9030DA
:1026000083168700831287143014E83083168900FC
:1026100083120915162B90308316870083128710BA
:102620003010E830831689008312091100340A142F
:102630008A140A1182078528B128D8281029372939
:1026400085299E29F2292D2A532A822AA02A662921
:10265000A82AB22A831606168312061E4C2B571977
:102660004A2B57158316861600308312861A0130BE
:10267000003A031D492B59085B02031C482B031D1C
:10268000452B5A0858020318482BD80A0319D90AAF
:10269000492B4B2B682B682B571D672B5711831623
:1026A000861600308312861A0130013C0319662B0E
:1026B0005D085902031C662B031D622B58085C023F
:1026C0000318662B58080319D903D803682B682B05
:1026D0008316200883125802031D742B83162108C9
:1026E000831259020319792B571C792BBB0198309F
:1026F000BA0059088316A100831258088316A00057
:1027000083128A150A16FE2B571EEC2B83162808F7
:102710000F3C0318D12BA801270CC600260CC500BE
:10272000C60CC50CC60CC50CC60CC50CC60CC50C1D
:102730000730C60545088312C400023083164607D9
:102740008312C5004508023C031CAE2B031DAC2BB5
:1027500044081B3C031CAE2BBD16AF2BBD124E080C
:10276000093C0319CD2B4E080D3C0319CD2BCE0887
:102770000319CD2B29308316D0000A1283121A2494
:102780000A167908FA007A084502031CCD2B031DAE
:10279000CC2B44087802031C49168316A701A60116
:1027A000E32B83121F151F19D32B1E08FA00831663
:1027B0001E08C3007A08C4004308A6070318A70A26
:1027C0004408A707A80A0830F80083121F08C73971
:1027D00078049F005712FA2B1F151F19ED2B831633
:1027E0001E088312C3000030F8001F08C7397804A0
:1027F0009F0057168A150A16112C47088316A50044
:10280000A5092830D5000A128312CA230A167808AF
:10281000CB00BC1C0F2CBC104130F8002A2D3C1DF5
:10282000152C3C114230F8002A2DBC1D1B2CBC116C
:102830004330F8002A2D3C1E212C3C124430F80075
:102840002A2DBC1E272CBC124530F8002A2DBD1C99
:10285000342C8316A51B322C8312BD100530F800D2
:102860002A2D83163D2C83128316A51F3D2C83121F
:10287000BD148530F8002A2D83168312471C432C83
:102880004230CD00452C2030CD00BC1F572C4708CE
:102890000139003A031D542CD608031D532CBC13D8
:1028A0000130F8002A2D562CE430D6005F2C471C4E
:1028B0005F2CE430D600BC178130F8002A2DD71CDD
:1028C000662CD7103C138230F8002A2D3C1F752C43
:1028D0008316A51C6D2CA519732C83123C13823012
:1028E000F8002A2D8316822C83128316A51C822CB5
:1028F000251D822CA51D822C83123C170230F80066
:102900002A2D83168312C6080319902C46088316B5
:10291000A5008312C60183162508F80083122A2D0C
:102920008316251EA32C831249080439003A031D7F
:10293000A02C4B1DA02C3C1349158230F8002A2DE9
:102940004915A52C8316831249118316A51EB72C91
:10295000831249082039003A031DB52CCB1EB52C33
:102960003C13C9168230F8002A2DC916831683122B
:102970003D1AC32C491EC32C4B1EC32C3C133D16C1
:102980008230F8002A2D41083F05003A0319F52C42
:102990008316A3012308073C031CF42C0130A40078
:1029A0002308F8000319D82C0310A40DF80BD42C1D
:1029B000831241083F0583162405003A0319F22CBF
:1029C0002408FF3A8312C1058316220EF700F03067
:1029D000F7057708803E2307013E073EF800831283
:1029E0002A2D8316A30ACA2C83123F08FF3A4105F9
:1029F000003A0319282D8316A3012308073C031C62
:102A0000272D0130A4002308F80003190B2D031013
:102A1000A40DF80B072D83123F08FF3A41058316DA
:102A20002405003A0319252D2408FF3A8312C10515
:102A30008316220EF700F030F70577082307013ED2
:102A4000073EF80083122A2D8316A30AFD2C831259
:0A2A50000030F8008A150A16162C53
:103000001F3083055730F700203084008001840A88
:10301000F70B0628F801F901FA01FB01FC01FD019B
:10302000FE015030F700A03084008001840AF70BC5
:103030001528A00184011F30830583161F149F14D7
:103040001F159F110C309900263098009030831284
:103050009800A801A901AA010130AB00AC01AD01A3
:10306000AE01F601FC015711D7118316A001A10191
:10307000A201A301A401A501831257128316A60180
:10308000A701A801A901AA01AB01AC01AD018312FE
:10309000D7128316B2018312D30114308316D600DF
:1030A0000A128A11831201230A168A153D10C601DD
:1030B0000730F700F71D6428073081018130840054
:1030C0000008C0390F388000640081308400000897
:1030D000C0397704800083161F149F101F159F119D
:1030E00083121F179F1783169F1783121F149412A2
:1030F0009030831687008700870030308312940059
:103100004030831694000030F80083121F08C7393E
:1031100078049F000A128A116F2B0A168A15013053
:103120008316D5000A128A118312CA230A168A1539
:10313000780FC9298316CE010230D0001630CF0097
:103140000A128A11831204240A168A1564000230B6
:103150008316CE00D0011E30CF000A128A118312CE
:1031600004240A168A15640004308316CE00D001A8
:10317000E430CF000A128A11831204240A168A1539
:10318000640006308316CE000130D0003130CF000D
:103190000A128A11831204240A168A1564000A305E
:1031A0008316CE000730D0002730CF000A128A11D4
:1031B000831204240A168A15640008308316CE0090
:1031C0000130D0007D30CF000A128A11831204240E
:1031D0000A168A1564001E308316CE000230D00015
:1031E0001630CF000A128A11831204240A168A1597
:1031F00064000C308316CE000130D0003130CF0097
:103200000A128A11831204240A168A1564000E30E9
:103210008316CE003530D000A430CF000A128A11B8
:10322000831204240A168A15640010308316D30012
:103230000430D4000A128A118312D9230A168A157F
:10324000640015308316D3005A30D4000A128A1154
:103250008312D9230A168A15640016308316D30008
:103260001430D4000A128A118312D9230A168A153F
:10327000640017308316CE000630D0008E30CF00A9
:103280000A128A11831204240A168A15640019305E
:103290008316D3003C30D4000A128A118312D9233A
:1032A0000A168A151A308316CE00D001CF010A12F1
:1032B0008A11831204240A168A1564001C308316AE
:1032C000CE00D001CF010A128A11831204240A16FB
:1032D0008A1520308316CE000230D000BC30CF00DB
:1032E0000A128A11831204240A168A1522308316C0
:1032F000CE00D0015B30CF000A128A118312042461
:103300000A168A1525308316D3000830D4000A1215
:103310008A118312D9230A168A1524308316D30002
:103320000430D4000A128A118312D9230A168A158E
:10333000640026308316CE00D0013230CF000A124E
:103340008A11831204240A168A1528308316D300A2
:103350003E30D4000A128A118312D9230A168A1524
:1033600029308316CE000330D0005230CF000A122D
:103370008A11831204240A168A152B308316CE0074
:10338000D001F030CF000A128A11831204240A16E9
:103390008A15D301FF30BF00C000C101831642105F
:1033A0008312D710C901CA01BD110730BE00033016
:1033B000D5009330D4003D17C9100630CE000A1254
:1033C0008A1136240A168A15CE01C8015710C20187
:1033D000E401E501AF01B00190308316870083124C
:1033E00007110A128A1198240A168A15FF308316CB
:1033F000C3008A11831200208A150A12CE260A16EB
:103400008B1683168C16C03083128B048316B3017F
:1034100001308312B1000C308316D5000A128A11D4
:10342000831251270A168A158316C30143080A120C
:103430008A118312AC220A168A158316C30AF70072
:10344000D5000A128A11831251270A168A151230E2
:1034500083164302031D162A8312BC12BB01983047
:10346000BA003D1290308316870083120710640063
:10347000BD1F3E2ABD130A12F72E0A166508640204
:103480000319FA2B0A12472F0A1678088316B1007F
:103490003108203C031D4F2A0130B200FB2BB2083B
:1034A0000319FB2B31080D3C031DBC2B03303202EA
:1034B000F83E0318BA2B083E8312892C8316BA2BC8
:1034C0008316BA2B83163808C5000A1283125B27AD
:1034D0000A16780E8316C400F030C4053908C500FA
:1034E0000A1283125B270A16780883164407B8006D
:1034F0003A08C5000A1283125B270A16780E831653
:10350000C400F030C4053B08C5000A1283125B27D3
:103510000A16780883164407B9003708563C031D7D
:10352000972A0A128312CE260A168316BA2B370858
:10353000573C031DA02A38088312C6008316BA2BF5
:10354000B50135082A3C031CB82B3508CC000330E4
:10355000CD000A128A118312C2270A168A1578082A
:103560000A128A1188200A168A15F8008316BC00F0
:1035700037083C02031DB62B3508CC000330CD00C4
:103580000A128A118312C2270A168A150130780797
:103590000A128A1188200A168A15F8008316BD00BF
:1035A0003508CC000330CD000A128A118312C227DD
:1035B0000A168A15023078070A128A1188200A161C
:1035C0008A15F8008316BE00BD080319B52B3D0B04
:1035D000052B3608573C031DF52A3208053C031D10
:1035E000F52A3E088400380880003E088400000860
:1035F000C3003708C600C7014308C800C9010A1242
:10360000831295270A16B42B83163D08023C031D2E
:10361000302B3608573C031D1A2B3208073C031D7C
:103620001A2B3E0884003908800001303E078400D0
:103630003808800001303E0784000008C3003E08BF
:1036400084000008C4003708C6004308C7004408C7
:10365000C800C9010A12831295270A16B42B8316D3
:103660003D08E03C0319B52B3D08E13C031D622BEE
:103670003608573C031D4B2B3208053C031D4B2BD2
:103680003E08D3003808D4000A128A118312D923C5
:103690000A168A1583163E08D5000A128A1183126B
:1036A000CA230A168A1578088316C3003708C6008D
:1036B000C7014308C800C9010A12831295270A16D8
:1036C000B42B83163D08E23C031DAB2B3608573C58
:1036D000031D862B3208073C031D862B01303E0755
:1036E000C300D3003808D4000A128A118312D923E8
:1036F0000A168A1583163E08D3003908D4000A1228
:103700008A118312D9230A168A15831601303E07BF
:10371000C300D5000A128A118312CA230A168A1519
:1037200078088316C4003E08D5000A128A11831255
:10373000CA230A168A1578088316C5003708C600FA
:103740004408C7004508C800C9010A12831295271A
:103750000A16B42B83163708C600C701C801C90171
:103760000A12831295270A168316B82BB50AA12AC6
:10377000BA2B8316B201FB2B01303202F73E03183D
:10378000FB2B093E8312952C83163108B6000230BC
:10379000B200FB2B83163108B7000330B200FB2BBD
:1037A00083163108B8000430B200FB2B83163108B1
:1037B000B9000530B200FB2B83163108BA00063081
:1037C000B200FB2B83163108BB000730B200FB2B85
:1037D00083163108BC000830B200FB2B8316310879
:1037E000BD000930B200FB2B83163108BE000A3041
:1037F000B200FB2B83168A1183122A2B8A1583169B
:103800003308FB3E0318812C053E8312A22C3C1C7E
:10381000122C3C100A128A1198240A168A158A1151
:10382000842B8A158316812C8A11FD2B8A15780822
:103830008316B4003408C3008A11831200208A154D
:103840008316B4080319312C421C312C5730C600A2
:10385000C7013408C800C9010A12831295270A1645
:103860008316812C0A128A1136240A168A158316A9
:10387000812C571C722C480DF700F70DF70DF8300E
:10388000F7057708013E0A128A1110210A168A15D7
:10389000DF3C0318722C01308316D6000230D700AB
:1038A0000A128A1183123D270A168A1510308400E5
:1038B00059088316CB00831258088316CA000A12CF
:1038C00083122A210A1604308316C3002030D50043
:1038D0000A128A11831251270A168A158316C30BFE
:1038E000662C83128316812C8316C601C701C8017A
:1038F0000130C9000A12831295270A168316812CFB
:103900008316B30A3308053C0319B3018312372A1F
:1039100063000A108A100A158207622A5E2A622A48
:10392000B92B622AB92BB92B602A0A108A100A1502
:103930008207C42BCA2BD02BD62BDC2BE22BE82BF7
:10394000EE2BF42B0A108A100A158207072C142C70
:06395000322C392C742C0E
:02400E00723FFF
:00000001FF
